:020000007C2B57
:10000800FF00030E8301AE000A08AF008A018B1CB3
:1000180010280130A3008B102F088A002E0E8300B1
:06002800FF0E7F0E09002F
:10002E007408F8027508031C750FF9027608031C94
:10003E00760FFA027708031C770FFB02F30D0730D9
:10004E00FC00730DF80DF90DFA0DFB0D7408731C01
:10005E003E28F8027508031C750FF9027608031C7A
:10006E00760FFA027708031C770FFB024B28F8076E
:10007E0075080318750FF90776080318760FFA0737
:10008E0077080318770FFB07F30DFC0B2828720D6A
:10009E00F80DF90DFA0DFB0D7408731C6428F802A7
:1000AE007508031C750FF9027608031C760FFA0209
:1000BE007708031C770FFB027128F80775080318E1
:1000CE00750FF90776080318760FFA0777080318E5
:1000DE00770FFB07F20D0730FC00720DF80DF90DCE
:1000EE00FA0DFB0D7408721C8A28F8027508031CA1
:1000FE00750FF9027608031C760FFA027708031CB7
:10010E00770FFB029728F80775080318750FF90784
:10011E0076080318760FFA0777080318770FFB0790
:10012E00F20DFC0B7428710DF80DF90DFA0DFB0D87
:10013E007408721CB028F8027508031C750FF902BA
:10014E007608031C760FFA027708031C770FFB0262
:10015E00BD28F80775080318750FF90776080318F8
:10016E00760FFA0777080318770FFB07F10D0730A4
:10017E00FC00710DF80DF90DFA0DFB0D7408711CD4
:10018E00D628F8027508031C750FF9027608031CB1
:10019E00760FFA027708031C770FFB02E328F807A5
:1001AE0075080318750FF90776080318760FFA0706
:1001BE0077080318770FFB07F10DFC0BC028700DA5
:1001CE00F80DF90DFA0DFB0D7408711CFC28F802E0
:1001DE007508031C750FF9027608031C760FFA02D8
:1001EE007708031C770FFB020929F8077508031817
:1001FE00750FF90776080318760FFA0777080318B4
:10020E00770FFB07F00D0730FC00700DF80DF90DA0
:10021E00FA0DFB0D7408701C2229F8027508031CD8
:10022E00750FF9027608031C760FFA027708031C85
:10023E00770FFB022F29F80775080318750FF907BA
:10024E0076080318760FFA0777080318770FFB075F
:10025E00F00DFC0B0C29701842297408F80775086C
:10026E000318750FF90776080318760FFA07770843
:08027E000318770FFB070800CD
:10028600FB09FA09F909F809F80A0319F90A031921
:08029600FA0A0319FB0A080033
:10029E00831203132230FC00F801F901FA01FB016D
:1002AE00FC03031985290310FB0CFA0CF90CF80C4E
:1002BE00F30CF20CF10CF00C031C5729FC03031980
:1002CE0077297408F80775080318750FF90776086B
:1002DE000318760FFA0777080318770FFB075B29C9
:1002EE007408F80775080318750FF90776080318D0
:0E02FE00760FFA0777080318770FFB07080042
:0C030C00831226088A00250882000800E1
:1003180083127408003A031DA6297508003A031DC4
:10032800A6297608003A031DA6297708003A031D76
:10033800A629FF30F000FF30F100FF30F2007F30D7
:10034800F3003F2A83120313FC01F71BFC0AFD018B
:10035800FB01FA01F901F8017308720471047004D1
:1003680003193A2A73087706A000A01BFD09F71F96
:10037800C829F409F509F609F709F40A0319F50A71
:100388000319F60A0319F70AF31FD529F009F10929
:10039800F209F309F00A0319F10A0319F20A031919
:1003A800F30A73087704A000A01BF6291720FC1B8A
:1003B800132AFD1F3A2AF009F109F209F309F00A94
:1003C8000319F10A0319F20A0319F30AF809F909DA
:1003D800FA09FB09F80A0319F90A0319FA0A0319B1
:1003E800FB0A3A2AF71F0D2AF31B072A7308FB009A
:1003F8007208FA007108F9007008F800F301F201B8
:10040800F101F001DD29F301F201F101F001F00A37
:100418000034F309F209F109F009FC17DA29F80A9E
:100428000319F90A0319FA0A0319FB0A740878026E
:10043800031DDD2975087902031DDD2976087A0276
:10044800031DDD2977087B02031DDD29FB01FA0165
:10045800F901F801F00A0319F10A0319F20A03195C
:10046800F30AF31FDD29A0012016FF34A0017C1C2C
:080478003E2A4321003E08006A
:1004800040308312F0001F30F100F201F301080048
:100490008312C203C2034208003C0318542AC20359
:1004A0000000000000004B2A0000000000000000D7
:0404B0000000080040
:1004B40001308312B1002708B0062B0884002708F6
:1004C400003A0319682A240880046A2A2D08800542
:1004D4002808C2004822B00931080319862A3108C5
:1004E4003005F000031D792A240880047B2A2D0896
:1004F4008005B10D311002302802C20048220000EC
:100504000000000000006E2A2708003A03198D2A13
:100514002D0880058F2A240880042808C200482258
:020524000800CD
:1005260083123008AB003108F0000130F200700889
:100536000319A12AF20D7210FF3E9B2A7208AA0027
:100546007209AC003208F1000130F000710803199D
:10055600B02AF00D7010FF3EAA2A7008A400F00918
:100566007008AD008030300784007208800470087F
:100576008005A70137080319C12AA709841327088C
:10058600003A0319C92A2D088005CB2A24088004BD
:100596004022E830F4000330F500F601F7014F2160
:1005A6007008B8007108B9007208BA007308BB0079
:1005B6003308F0003408F1003508F2003608F3007D
:1005C600F00DF10DF20DF30D7010F00DF10DF20DB1
:1005D600F30D70100A30F400F501F601F7014F2112
:1005E6007008BC007108BD007208BE007308BF0029
:1005F6007008F4007108F5007208F6007308F70039
:100606003808F0003908F1003A08F2003B08F30018
:100616008C217008C0007108C1007108F400F50152
:100626007408750403191A2B0230F0006F2B40086A
:10063600A8003C08F4003D08F5003E08F6003F0817
:10064600F7003808F0003908F1003A08F2003B08D4
:10065600F3008C217808F0007908F1007A08F2009E
:100666007B08F3007008B8007108B9007208BA0078
:100676007308BB003C08F5003D08F6003E08F7008D
:100686003F08F800F80CF70CF60CF50CF813781B7D
:10069600F81780307806F400803073067402031D64
:1006A6005E2B72087702031D5E2B71087602031D0E
:1006B6005E2B700875020318612BA80A2808F10042
:1006C600F10CF1137108A9000730710203186E2BA3
:0A06D6000130F0006F2BF001080066
:1006E00086218A110A128000840AA50A0319A60A23
:0806F000F003031D702B08004C
:1006F8008312A101A201A301713083168F009F010B
:100708000730831299009F01D0308B001C3083166C
:100718008500831285018316810104309500053018
:100728008312B0000430B1000530B2006030B3006D
:100738000930B400B501B601B70193220230FB00BD
:100748000430FC00BA30FD00FD0BA82BFC0BA82BD5
:10075800FB0BA82B000023080319EF2B851403308B
:10076800FB000830FC007730FD00FD0BB92BFC0BBB
:10077800B92BFB0BB92BA201033022020318DD2B86
:10078800A1010E3021020318DB2B2108F13EF000F5
:1007980003300318013EF1007008A5007108A60097
:1007A80086218A110A12B0005A22A10AC52BA20A70
:1007B800C02B85100B30FB002630FC005D30FD009F
:1007C800FD0BE42BFC0BE42BFB0BE42B00000000DF
:0A07D800A30163000000AF2BF02B1B
:1007E20053347A3465347A3461346D345F3474341A
:0E07F2006134723475346C346A34213400344E
:02400E00D40FCD
:00000001FF
